:100000006EC00AC92EC985C084C084C082C081C0A8
:1000100080C07FC07EC093C37CC07BC07AC079C0E3
:1000200078C077C022C375C074C073C072C071C07D
:1000300070C06FC0B1C52FC61DC838C61BC81AC84E
:1000400019C818C817C816C815C814C813C84CC68C
:1000500011C89FC62CC70EC8CDC7DEC7FBC741203D
:10006000000042C80000461C40004CBEBC205A0E96
:100070001BCA749DC5AE3DCCCCCD3C23D70A38D12C
:10008000B717322BCC7724E695950A4FB11F063966
:10009000652C033AA23B593C1EBAE03D633BF43E5B
:1000A00075FF4E3F3172113F800000000540B504DE
:1000B000F441A0000141E2463241A0000040E24686
:1000C000303F8000000541778C4F40C32CE2411740
:1000D000BF24C1A48DD9C0E1D8A1C05B678211241F
:1000E0001FBECFEFD4E0DEBFCDBF11E0A0E0B1E096
:1000F000E8EEFCE102C005900D92A035B107D9F7FA
:1001000011E0A0E5B1E001C01D92AA3DB107E1F701
:10011000F8C076CF1F920F920FB60F9211248F93D3
:10012000AF93BF93EF93FF9385B1836085B9E8E701
:10013000F1E0A9E0B0E084E0182E9BDDFF91EF91A3
:10014000BF91AF918F910F900FBE0F901F90189598
:1001500085E08093690083E08DBB84E08093680034
:1001600080E480936D0084B1836084B985B183603D
:1001700085B978940895DC01CB012FEB3EE04CE982
:100180005EE3BC01CD01DADADC01CB01BC01CD01BB
:100190002CDADC01CB01BC01CD0144DADC01CB015E
:1001A000BC01CD0108959F92AF92BF92CF92DF9292
:1001B000EF92FF920F931F93CF93DF93CDB7DEB7EC
:1001C00060970FB6F894DEBF0FBECDBF6B017C0108
:1001D000909073015E010894A11CB11C80E1F501AF
:1001E00011928A95E9F780915901882339F0C70166
:1001F000B601C1DF6B017C019090680120916F0115
:10020000309170014091710150917201C701B601A6
:1002100095DA6B017C01850120916D014091C80147
:100220005CD931E0F5018181882389F090E3F80100
:10023000E30FF11D80818D3211F0803209F490833B
:100240003F5FF801E30FF11D8081882381F7409122
:10025000C801431750F4FE0132969EE081818193DC
:10026000915097FFFBCF3150F4CF20E030E040E0D9
:1002700050E0C701B601E0D9882311F480E28983F8
:1002800020E030E040E050E0C701B601D5D9882336
:1002900014F48DE2898320E030E040E050E0C701B3
:1002A000B601CDD9181614F48BE28983CE010196DC
:1002B0000ED2892D05D260960FB6F894DEBF0FBE20
:1002C000CDBFDF91CF911F910F91FF90EF90DF9005
:1002D000CF90BF90AF909F9008958BE591E0F7D1BC
:1002E0008091780190917901A0917A01B0917B0180
:1002F000BC01CD0197D9DC01CB01BC01CD0153DF9D
:100300000895C9EED4E0DEBFCDBF40E050E660E026
:1003100070E039E0CA010197F1F7315037FFFACFA9
:10032000109259013ED114DFC4D1E9D180E091E0AF
:100330006DD18DE050D10BE1009383011BE510934B
:10034000840181E3F82EF09285018BE4809386018D
:100350001092870100935B0110935C0190E39093EE
:100360005D0190935E018BE380935F019093600148
:100370009093610188E48093620110926301A1E08F
:10038000B0E05EDC802D982FA2E0B0E059DC802D3B
:10039000890FA3E0B0E054DC902D980FA4E0B0E00A
:1003A0004FDC802D890F863009F07FC0A5E0B0E0DA
:1003B00047DC802D992780937401863010F01092CD
:1003C0007401A6E0B0E03CDC802D992780935901B0
:1003D000823010F010925901A7E0B0E031DC802D9E
:1003E00080936901A8E0B0E02BDC802D80936D0143
:1003F000E8E7F1E0A9E0B0E084E0182E29DCEFE6C0
:10040000F1E0ACE1B0E0182E23DCAFE0B0E018DCA6
:10041000802D80937301A0E1B0E012DC802D8093E9
:100420006801A1E1B0E00CDC802D8093C801A2E15D
:10043000B0E006DC802D80938001A3E1B0E000DC19
:10044000802D80936A01A4E1B0E0FADB802D8093D7
:100450007F01A5E1B0E0F4DB802D80937701A6E178
:10046000B0E0EEDB802D80938101A7E1B0E0E8DB16
:10047000802D80937501A8E1B0E0E2DB802D8093B0
:100480005A01A9E1B0E0DCDB802D80936E01AAE186
:10049000B0E0D6DB802D80938201ABE1B0E0D0DB11
:1004A000802D809358016DD12EC020E030E0A9014D
:1004B000B90182E739D3A1E0B0E090E0092ECDDBAD
:1004C000A2E0B0E081E0082EC8DBA3E0B0E082E06B
:1004D000082EC3DBA4E0B0E083E0082EBEDB098376
:1004E00081E58A830B8382E58C830D831E8388E3F9
:1004F0008F8386E7888709871A87FB868C879D8785
:10050000CE010196E4D0E9DEDDD680916B019091B9
:100510006C01892B09F425D2809174018530C1F1D9
:10052000C0907801D0907901E0907A01F0907B0141
:100530008091640190916501A0916601B09167017D
:10054000C816D906EA06FB0629F4C114D104E10451
:10055000F104F1F48E01025F1F4F20E130E0A801A9
:10056000C701B601E7D6C80151D08DE034D0B5DE61
:100570008091780190917901A0917A01B0917B01ED
:100580008093640190936501A0936601B093670125
:1005900090917E0180917601981709F4B5CF79D5B5
:1005A000B3CF10927E011092760140E450E060E0FB
:1005B00070E088E891E098D6519A1092C5008FE3D8
:1005C0008093C40088E98093C10086E08093C200D4
:1005D0008091C6000895982F8091C00085FFFCCFC0
:1005E0009093C600089580917E01E82FFF27E85779
:1005F000FE4FE0818F5F80937E01803411F4109272
:100600007E018E2F992787FD90950895EF92FF9296
:100610000F931F93CF93DF937C0100E010E0FC0168
:1006200080818823D9F0F801EE0DFF1D8081E8015B
:1006300021968B3161F48CE3CEDF85E4CCDF83E55A
:10064000CADF83E4C8DF8EE3C6DF8E0102C08E01FD
:10065000C2DFCE0DDF1D8881882329F7DF91CF917E
:100660001F910F91FF90EF9008951F920F920FB678
:100670000F9211248F93EF93FF9380917601E82FCF
:10068000FF27E857FE4F8091C60080838091760156
:100690008F5F8093760180917601803411F41092FF
:1006A0007601FF91EF918F910F900FBE0F901F90E9
:1006B000189584B18C6284B92A9A8DE58CBD089511
:1006C0002A988EBD0DB407FEFDCF2A9A08951F9378
:1006D000CF93DF93EC0110E08881882361F0FE0165
:1006E000E10FF11D8081ECDF1F5FFE01E10FF11DC5
:1006F00080818823A1F7DF91CF911F91089587B161
:10070000807E87B988B18F6188B9809181008C60C3
:100710008093810084E690E0909389008093880024
:10072000B19A80916F00826080936F0081E090E0C9
:1007300090936C0180936B011092C90108951F92F0
:100740000F920FB60F9211248F939F9380916B019C
:1007500090916C01019790936C0180936B01809153
:100760006B0190916C01892B29F480916F008D7F32
:1007700080936F009F918F910F900FBE0F901F90ED
:100780001895CF93DF93CDB7DEB723970FB6F894C4
:10079000DEBF0FBECDBF80917401992782309105D5
:1007A00009F45AC0833091052CF4009759F0019751
:1007B00071F1CEC08330910509F473C0049709F438
:1007C00095C0C6C0809180014AE050E0BE016F5FD5
:1007D0007F4F992790D58091800199818A3030F49C
:1007E00080E3809360019093610105C09093600164
:1007F0008A818093610180916A014AE050E0BE01E4
:100800006F5F7F4F992777D580916A0193C0809160
:100810007F014AE050E0BE016F5F7F4F99276BD5A3
:1008200080917F0199818A3030F480E38093600168
:100830009093610105C0909360018A81809361016A
:10084000809177014AE050E0BE016F5F7F4F9927AA
:1008500052D5809177016EC0809181014AE050E0CD
:10086000BE016F5F7F4F992746D5809181019981A5
:100870008A3030F480E3809360019093610105C079
:10088000909360018A8180936101809175014AE0B3
:1008900050E0BE016F5F7F4F99272DD58091750184
:1008A00049C080915A014AE050E0BE016F5F7F4F1E
:1008B000992721D580915A0199818A3030F480E3BB
:1008C000809360019093610105C0909360018A81DB
:1008D0008093610180916E014AE050E0BE016F5F3C
:1008E0007F4F992708D580916E0124C080918201A5
:1008F0004AE050E0BE016F5F7F4F9927FCD48091A2
:10090000820199818A3030F480E380936001909372
:10091000610105C0909360018A818093610180919B
:1009200058014AE050E0BE016F5F7F4F9927E3D442
:100930008091580199818A3030F480E380935D0181
:1009400090935E0105C090935D018A8180935E0162
:1009500023960FB6F894DEBF0FBECDBFDF91CF91C7
:10096000089586B18F718095282F3327C9018F7123
:100970009070892B19F41092C901089520FF22C0AC
:1009800088EC90E090936C0180936B0180916F00F4
:10099000826080936F00809174018F5F80937401F7
:1009A000863010F010927401ECDE83E891E08FDE67
:1009B00080917401853009F090DCA5E0B0E0809171
:1009C000740123C021FF24C088EC90E090936C0157
:1009D00080936B0180916F00826080936F008091A3
:1009E0005901882319F01092590103C081E08093C6
:1009F000590183E891E06BDE80917401853009F044
:100A00006CDCA6E0B0E080915901082E26D908954B
:100A100022FF16C023FF14C088EC90E090936C0175
:100A200080936B0180916F00826080936F001092C1
:100A300078011092790110927A0110927B01089549
:100A400024FF14C088EC90E090936C0180936B01BC
:100A500080916F00826080936F00109278011092F5
:100A6000790110927A0110927B012DC022FF2DC0D6
:100A70002091C9012A3018F488EC90E002C08AE085
:100A800090E090936C0180936B0180916F00826085
:100A900080936F002B3018F42F5F2093C90112D47C
:100AA0008091780190917901A0917A01B0917B01B8
:100AB0000196A11DB11D8093780190937901A093B7
:100AC0007A01B0937B0107D4089523FF2CC02091B5
:100AD000C9012A3018F488EC90E002C08AE090E066
:100AE00090936C0180936B0180916F008260809382
:100AF0006F002B3018F42F5F2093C901E3D380914E
:100B0000780190917901A0917A01B0917B010197D0
:100B1000A109B1098093780190937901A0937A019A
:100B2000B0937B01D8D30895CF92DF92EF92FF92DA
:100B30000F931F93CF93DF93CDB7DEB7A3970FB675
:100B4000F894DEBF0FBECDBF6A0189013BE1398356
:100B50002BE52A8350E35B839AE79C831D823E83C7
:100B60002F8341E3488796E399879BE39A875B87C6
:100B700096E79C873D872E874F87988B198A992700
:100B8000AA27BB27FC01E356F040E531F10508F048
:100B900071C2E65EFF4F09946115710509F5C60142
:100BA000AA2797FDA095BA2FBC01CD013BD57B01AB
:100BB0008C01D7FE07C020E030E040E857E405D4C0
:100BC0007B018C01BE016E5D7F4F8AEC91E049D6BE
:100BD000DC01CB019C01AD01C801B701F6D343C0D4
:100BE0006130710509F050C0C601AA2797FDA09594
:100BF000BA2FBC01CD0116D57B018C01D7FE07C0F1
:100C000020E030E040E857E4E0D37B018C01BE01F6
:100C10006E5D7F4F8AEC91E024D6DC01CB019C0114
:100C2000AD01C801B701D1D37B018C01609178017E
:100C30007091790180917A0190917B0197FF04C0B6
:100C40006D5F7F4F8F4F9F4F32E0959587957795DA
:100C500067953A95D1F7E6D4DC01CB019C01AD0153
:100C6000C801B701F4D3DC01CB0180936F019093ED
:100C70007001A0937101B0937201EFE6F1E0ACE175
:100C8000B0E084E0182EF5D780E1EAECF1E01192B3
:100C90008A95E9F7EBC16530710508F0EBC1609307
:100CA0006D01A8E0B0E0062ED8D7E0C1611571054E
:100CB00039F4809169018D7F8093690180E309C0D7
:100CC0006130710539F48091690182608093690116
:100CD00085E38B83A7E0B0E080916901082EBDD742
:100CE000CE010196F4DCC2C16230710559F1633066
:100CF000710538F46115710559F061307105A9F07D
:100D0000D4C06330710559F164307105A9F1CDC0CB
:100D1000C092800100936A01A2E1B0E00C2C9DD743
:100D2000A3E1B0E080916A01BEC0C0927F01009350
:100D30007701A4E1B0E00C2C90D7A5E1B0E0809160
:100D40007701B1C0C092810100937501A6E1B0E0C6
:100D50000C2C83D7A7E1B0E080917501A4C0C092AC
:100D60005A0100936E01A8E1B0E00C2C76D7A9E1FE
:100D7000B0E080916E0197C0C0928201009358014B
:100D8000AAE1B0E00C2C69D7ABE1B0E0809158014A
:100D90008AC010927401A5E0B0E010E0012E5DD78A
:100DA00010935901A6E0B0E0012E57D710936901C6
:100DB00000E30B83CE0101968ADC0B87CE010696F9
:100DC00086DCA7E0B0E080916901082E46D781E07B
:100DD00080936D01A8E0B0E0082E3FD78DEC9CEC2D
:100DE000ACECBDE380936F0190937001A09371010F
:100DF000B0937201EFE6F1E0ACE1B0E084E0182ED0
:100E000038D786E480937301AFE0B0E0082E25D791
:100E10008DE480936801A0E1B0E0082E1ED797E032
:100E20009093C801A1E1B0E0092E17D7109380017B
:100E3000A2E1B0E0012E11D710936A01A3E1B0E066
:100E4000012E0BD72AE120937F01A4E1B0E0022E0E
:100E500004D710937701A5E1B0E0012EFED68EE015
:100E600080938101A6E1B0E0082EF7D6909375013A
:100E7000A7E1B0E0092EF1D610935A01A8E1B0E045
:100E8000012EEBD68FE080936E01A9E1B0E0082E31
:100E9000E4D620938201AAE1B0E0022EDED6809350
:100EA0005801ABE1B0E0082ED8D66BDCDFC08FE094
:100EB00091E0ACDB8DE08FDB8EE191E0A7DB8091F0
:100EC0007401805D88DB8DE086DB86E291E09EDB4D
:100ED0008091690199278270907095958795805DC2
:100EE0007ADB8DE078DB8EE291E090DB82E1E82E28
:100EF000F12CEC0EFD1E80916F0190917001A0917C
:100F00007101B0917201870125E048E0BC01CD017B
:100F1000E4D2C7017BDB8DE05EDB8EE391E076DB24
:100F2000809169018170805D56DB8DE054DB80919A
:100F3000740199278230910551F1833091052CF489
:100F4000009749F00197A9F095C08330910569F1A8
:100F50000497C9F18FC0809180014AE050E0B70149
:100F60009927C9D1C70152DB8CE235DB80916A0138
:100F700037C080917F014AE050E0B7019927BBD18B
:100F8000C70144DB8CE227DB8091770129C0809187
:100F900081014AE050E0B7019927ADD1C70136DBA6
:100FA0008CE219DB809175011BC080915A014AE0E7
:100FB00050E0B70199279FD1C70128DB8CE20BDBFA
:100FC00080916E010DC0809182014AE050E0B7012E
:100FD000992791D1C7011ADB8CE2FDDA8091580183
:100FE0004AE050E0B701992786D1C7010FDB8DE0B9
:100FF000F2DA40C06115710529F4C0927301AFE0C7
:10100000B0E007C06130710589F5C0926801A0E1C8
:10101000B0E00C2C22D62AC06115710539F48091FC
:1010200069018E7F8093690180E309C06130710599
:1010300039F48091690181608093690181E38B8734
:10104000A7E0B0E080916901082E07D6CE01069690
:101050003EDB2BCFCB0102970F9760F46093C80162
:10106000A7E0B0E080916901082EF7D583E891E010
:101070002EDB33D9A3960FB6F894DEBF0FBECDBFDB
:10108000DF91CF911F910F91FF90EF90DF90CF9064
:101090000895A9DAA82F80915101992782309105EE
:1010A00059F1833091052CF4009771F00197E9F024
:1010B00008958430910509F465C084309105DCF110
:1010C000059709F480C008959093530180935201CD
:1010D000909355018093540190935701809356014A
:1010E000AB3109F098C081E004C0AB3509F068C0AD
:1010F00082E08093510108958A2F80538A30B0F4A2
:101100002091520130915301C90163E0880F991F6A
:101110006A95E1F7820F931F820F931F8A0F911D2B
:10112000C09790935301809352010895AB3309F017
:1011300043C083E0DECF8A2F80538A30B0F4209101
:10114000540130915501C90153E0880F991F5A95F8
:10115000E1F7820F931F820F931F8A0F911DC09793
:1011600090935501809354010895AE3239F485E08F
:1011700080935101A093CA0181E033C0AB33E1F405
:1011800084E0B7CF8A2F80538A30B0F42091560183
:1011900030915701C90143E0880F991F4A95E1F743
:1011A000820F931F820F931F8A0F911DC0979093F8
:1011B00057018093560108958A2F80548F33C0F0D1
:1011C00010925101089580915001803168F4A0334C
:1011D00058F0AA3348F4E82FFF27E653FE4FA083C8
:1011E0008F5F8093500108958A2F80548F3388F445
:1011F00010925101209156013091570140915401B4
:101200005091550160915201709153018A2F8CDCED
:1012100008951092510108950F932F939F939FB7B4
:101220009F9325B191E0292725B9062D29B12C706E
:10123000003019F4243071F00EC0083019F42C304D
:1012400049F009C0043019F4203021F004C02830DE
:1012500009F001C0622E9F919FBF9F912F910F9126
:1012600018950F932F939F932FB72F9325B192E04B
:10127000292725B9062D29B12C70003049F42830D2
:10128000D9F4112491E0291A31084108510813C0FA
:10129000083049F4203081F4112491E0290E311CEA
:1012A000411C511C08C0043019F42C3021F004C03A
:1012B000243009F001C0622E9F919FBF9F912F9112
:1012C0000F911895209278013092790140927A011D
:1012D00050927B01089520907801309079014090E0
:1012E0007A0150907B010895DC0101C06D9341505B
:1012F0005040E0F70895FB019F01E8944230BCF0B4
:101300004532ACF44A3029F497FB1EF49095819550
:101310009F4F642F7727B2D4805D8A330CF0895DAC
:101320008193CB010097A9F716F45DE251931082E7
:10133000C9013AC0FA01CF93FF93EF9322303CF1F9
:1013400025322CF5C22FE894CA3049F497FB3EF4BD
:1013500090958095709561957F4F8F4F9F4F2C2F63
:10136000332744275527FF93EF939CD4EF91FF91A8
:10137000605D6A330CF0695D6193B901CA01605028
:1013800070408040904059F716F4CDE2C19310822E
:101390008F919F91CF9108C07AE0979F902D879F62
:1013A000802D910D11240895DC01FC010190002095
:1013B000E9F73297AE17BF0730F47C9160817083F4
:1013C00031976D93F7CF08955058192E77D101D0EA
:1013D0005AC1BA176207730784079507B1F188F4F9
:1013E0000EF410940B2EBA2FA02D062E622F202D56
:1013F000072E732F302D082E842F402D092E952F68
:10140000502DFF275523B9F0591B49F0573E98F04E
:10141000469537952795A795F0405395C9F776F0EF
:10142000BA0F621F731F841F30F4879577956795F5
:10143000B795F040939517FA0F2E0895BF1BBB2761
:10144000BA0B620B730B840BF6CFDEF663C136D199
:1014500001D019C1552359F0992369F09F575F575F
:10146000951B33F442F4903811F4915805C023C110
:1014700091589F3F09F44EC1BB271124621773078F
:10148000840730F4660F771F881FBB1F915098F3B5
:1014900011D00F920FD00F920DD0A0E8261737076A
:1014A00048071B0609F0A048BA2F602D7F918F9145
:1014B00000240895A0E80024621773078407B1058B
:1014C00028F0621B730B840BB1090A2A660F771F81
:1014D000881FBB1FA69581F70895DF93CF931F93B5
:1014E0000F93E8018C01000F111F1F3F31F49EE4A0
:1014F00081E499938993999371C04F9399231AF436
:101500000DE209939F77022F03959F938F937F930B
:101510006F93622F77278827992784D09068AC0132
:101520009B0191E480E27727662750D15FEF4FEF70
:10153000F3D02F913F914F915F9147DF102F0130F2
:1015400009F4002751E440E233272227621773078A
:10155000840795071CF07BDF1395F4CF9F938F933F
:101560007F936F9342D0562F505D59935BD02F914C
:101570003F914F915F9128DF905851E440E233272B
:101580002227DCD0101711F45EE259931A9531F737
:1015900018825F91EF91FF91FF93EF93452F4423C2
:1015A00012F440954395CE01BF01861B970B142F73
:1015B000181B90E284179CF455236AF0219631960B
:1015C000E40FF11D83955A9152938A95E1F7929316
:1015D0001A95E9F704C099931A95E9F718828F9143
:1015E0009F918C01CF91DF91089597FB73D09F3726
:1015F00038F0FEE9F91B982F872F762F6B2F05C047
:1016000086C09695879577956795F150D0F73EF40B
:1016100090958095709561957F4F8F4F9F4F08955E
:10162000E89403C097FB0EF4F3DFB62F672F782FF3
:10163000892F9EE9002427C00ED05EF004C00BD095
:1016400026F001C008D019F020F48FEF089580E053
:10165000089581E0089597FB092E052600F8689407
:1016600030D0E89407FC07C062177307840795071A
:1016700021F008F400940794989408959A95BB0F6C
:10168000661F771F881F11249923A1F08823B2F7C2
:101690009F3F59F0BB0F48F421F4002011F460FF84
:1016A00004C06F5F7F4F8F4F9F4F881F979587951F
:1016B00097F908952CC09FEF80EC0895052E092618
:1016C00007FA440F551F5F3F79F0AA27A51708F0C6
:1016D00051E04795880F991F9F3F31F0BB27B917FD
:1016E00008F091E0879508959F919F911124E3CF91
:1016F00097FB880F991F9F3F31F0BB27B91708F060
:1017000091E0879508959F919F911124D4CF6627EA
:101710007727882799270895EBDF992359F0AA277F
:10172000940FA51F43F032F04FEF50E09417A50738
:1017300014F4A9CFECCF0EF09FC199C1BFDF01D047
:10174000A2CF992339F0552329F09F575F57950F62
:1017500013F49AF1DFCF91589F3FE1F3629FA12DDF
:101760000F92BB27639FA00DB11DEE27729FA00DA6
:10177000B11DEE1FAF93AA27649FB00DE11D739FAB
:10178000B00DE11DAA1F6627829FB00DE11DA61FA7
:101790005527749FE00DA11D551F839FE00DA11DCE
:1017A000561F849FA00D511D852F7A2F6E2F1F90DD
:1017B0000F9088231AF4939539F47DCF000C111CF7
:1017C000BB1F661F771F881F012808953CD038F083
:1017D0002ED060F186F021F436D009F03EF56BCFC3
:1017E0005F934F933F932F937CD12F913F914F91D4
:1017F0005F91A4DFECC027D098F389F00894E795B7
:10180000D901AA2329F4AB2FBE2FF85FD0F3E8CF7C
:10181000FF5F30F7A695E0F7F73908F309F09F77F7
:101820009F939F77DDDFEF91E0789E270895E894FE
:10183000FC01EE0FFF1F30966105710519F0F3955D
:10184000F14097FB0895E894FA01EE0FFF1F3096E0
:101850002105310519F0F395F14057FB08957727DD
:101860006627B0D0C82FD92F7F936F939D2E8C2ED3
:1018700009910032E9F30930D9F30637C9F30C3086
:10188000B9F30A30A9F30D3099F352D06ED0EEF1CE
:10189000C7DE17FB97F9C92ED82EE72EF62E88271C
:1018A0000062053651F4099143D04AD0992319F0CA
:1018B00017FD3CC035C017FD8195EEE5F0E0182F0F
:1018C0009C2D8D2D7E2D6F2D9F779817870776077E
:1018D0006105D9F01A0D3AF411957896912F9B195C
:1018E000973224F504C0912F9B0D9732CCF49C2D98
:1018F000112359F0159538F4AED0EF93FF931EDF06
:10190000FF91EF91F5CF3496F3CFEF91FF91E03057
:10191000EF0711F081929082ECE0CDB7DEB77BC18A
:101920009C2D9F678FE77FEF6FEFEFCFF0DEEDCF5E
:1019300011270B3219F00D3211F410680991089536
:1019400088279927003384F011F415FF09C00A3362
:101950005CF41062992321F41FDD0F70800F911D3C
:101960009D2E8C2E0991EECF08956894D0DEBB2475
:10197000BA94AA240E3229F416FD23C01064FEF096
:101980001CC00033F4F019F4E89415FF11C00A33B9
:10199000C4F410629F307CF4B394E8945527442734
:1019A00033272AE0F7D00F70600F711D811D911D44
:1019B00016FDAA9402C016FFA3949D2E8C2E0991A9
:1019C000D9CF0895AA27BB27FF91EF9108C1092E0F
:1019D00099234AF052E441EB32E7683173078407F8
:1019E000950758F068CE9F7752E44EEA3CEA60359E
:1019F00073078407950708F08ACE0F925FE348EBE0
:101A00003AEA2BE39BDEFF92EF92DF92CF9250E017
:101A10004CE090D0EEE8F0E034D05F2D4E2D3D2D1F
:101A20002C2DCF90DF90EF90FF90FEE94595441F5D
:101A3000551FF51B5527406804C0469537952795D7
:101A40005795FA95D2F7452F550F550B65DE0F9038
:101A500007FC06C00895559145913591259108954B
:101A60009B01AC019FE380E877276627F0CC9FEFCE
:101A700080E870E060E008959FE780E870E060E053
:101A80000895FF92EF92DF92CF92BF926B017C019B
:101A9000B59015D0B590BB2061F09F938F937F9345
:101AA0006F93B601C7010BD02F913F914F915F917A
:101AB000CEDCBF90CF90DF90EF90FF900895CBDF0A
:101AC00002C09601A701EF93FF9338DEFF91EF91DB
:101AD000C2DFEF93FF9379DCFF91EF91BA9489F71E
:101AE000089597FDE8CD04DE992309F4E4CDFF9233
:101AF000EF92DF92CF92C92E9FE38F77ECEAF0E06E
:101B0000C0DF0C2CC92ED82EE72EF62E602D6E5776
:101B1000770B872F972F86DD5FE341E332E728E1DC
:101B20000DDE5C2D4D2D3E2D2F2DCF90DF90EF90B3
:101B3000FF904BCCDDDDCF93DF93D52FC42F5527FE
:101B40004427332722279923D9F09F37C8F0F92F4C
:101B50009ADD592F482F372F262FF63968F445DDA7
:101B600061DDC030CD0721F0699379938993999312
:101B70009058DF91CF9129CC99278827772766271E
:101B8000C030CD0721F02993399349935993DF91C0
:101B9000CF9179CD629FD001739FF001829FE00DBC
:101BA000F11D649FE00DF11D929FF00D839FF00DDC
:101BB000749FF00D659FF00D9927729FB00DE11D88
:101BC000F91F639FB00DE11DF91FBD01CF01112465
:101BD00008952F923F924F925F926F927F928F92D1
:101BE0009F92AF92BF92CF92DF92EF92FF920F93AC
:101BF0001F93CF93DF93CDB7DEB7CA1BDB0B0FB6B6
:101C0000F894DEBF0FBECDBF09942A883988488872
:101C10005F846E847D848C849B84AA84B984C88408
:101C2000DF80EE80FD800C811B81AA81B981CE0FFF
:101C3000D11D0FB6F894DEBF0FBECDBFED010895E4
:101C4000F999FECFB2BDA1BDF89A119600B40895DE
:101C5000F7DF01921A94E1F70895F999FECFB2BD2A
:101C6000A1BD00BC11960FB6F894FA9AF99A0FBE6E
:101C700008950190F2DF1A94E1F70895AA1BBB1BA7
:101C800051E107C0AA1FBB1FA617B70710F0A61B7C
:101C9000B70B881F991F5A95A9F780959095BC019D
:101CA000CD010895A1E21A2EAA1BBB1BFD010DC098
:101CB000AA1FBB1FEE1FFF1FA217B307E407F507FC
:101CC00020F0A21BB30BE40BF50B661F771F881FD8
:101CD000991F1A9469F760957095809590959B016E
:081CE000AC01BD01CF01089524
:101CE800424F422D34205345492056312E3400426C
:101CF8004F422D34205345492056312E34004D6F24
:101D08006465203D2000466F6E74203D20005363BB
:101D1800616C6520666163746F72203D20005669AE
:101D280064656F205374616E64617264203D2000A5
:00000001FF
